:100000000C9448000C9465000C9465000C946500F9
:100010000C9465000C9465000C9465000C946500CC
:100020000C9465000C94B7000C9465000C9465006A
:100030000C9465000C9465000C9465000C946500AC
:100040000C9465000C9428030C94F3010C94AF01FC
:100050000C949A010C9465000C9465000C94650056
:100060000C9465000C9465006374726C5F616C6C39
:100070006F6328256429206964783D25640A007E21
:100080000E0E0E0E1B1B1C0E1B1B7E0E0E0E0E00EC
:1000900011241FBECFEFD4E0DEBFCDBF11E0A0E042
:1000A000B1E0E8E9F9E202C005900D92A231B10792
:1000B000D9F713E0A2E1B1E001C01D92A433B1076A
:1000C000E1F70E9470000C94CA140C940000809117
:1000D00012010895A8950E947C030E947210089551
:1000E000F894A8950E9450010E94EE020E943E0FD3
:1000F0008FEF80931001409A0E947601789480E0FF
:1001000090E060E040E050E00E94C61080E090E0A7
:100110000E94750F0E94240D0E9494020E9477088D
:100120000E946A00F9CF909112019817F1F0963071
:10013000E1F0953011F48630C1F4809312010E94F1
:10014000C60480911201853029F480E060E245E028
:100150000E946D1180911201863029F480E060E2E6
:1001600046E00E946D1181E0089580E008951F929D
:100170000F920FB60F9211248F939F93AF93BF935B
:1001800080912A03882329F080912A03815080934B
:100190002A0380911301882329F581E080931301BC
:1001A0007894809114018F5F8093140180911401E1
:1001B00090E083709070892B99F480912603909140
:1001C0002703A0912803B09129030196A11DB11D19
:1001D0008093260390932703A0932803B0932903C9
:1001E00010921301BF91AF919F918F910F900FBE0D
:1001F0000F901F90189510922603109227031092CB
:10020000280310922903E0E7F0E010821092B0007A
:1002100082E08093B1008081816080830895EF92B5
:10022000FF920F931F932091260330912703409153
:100230002803509129037C0100E010E0E20EF31E38
:10024000041F151F02C00E946A00C801B7010E9466
:1002500088118823C1F31F910F91FF90EF900895AB
:10026000EF92FF920F931F93209126033091270363
:1002700040912803509129037C0100E010E0E20E38
:10028000F31E041F151F01C0A895C801B7010E94E5
:1002900088118823C9F31F910F91FF90EF90089563
:1002A000EAEFFFE39491892F81508E3F10F49093F1
:1002B00066000895ECEFFFE3259135914591549147
:1002C0005070B901CA010895EFEFFFE3E4918E2F5A
:1002D0000895F8942CE088E190E00FB6F894A89582
:1002E000809360000FBE20936000FFCF1092160134
:1002F00080911601E6E1F1E08293808180933001E4
:100300008091300180932F01519A5098599A589AB0
:100310005A9882E08093C0001092C5008FE08093CD
:10032000C40086E08093C2008CEF8093C10080E01F
:1003300090E008951F920F920FB60F9211248F93A1
:100340001092160180911601809315015A988091A0
:10035000C6008F910F900FBE0F901F9018951F929F
:100360000F920FB60F9211248F939F93EF93FF93E9
:1003700090912F0180913001981731F48091C10044
:100380008F7D8093C10026C05A9A8091390187FFE2
:1003900009C0809139018F77809339018091C10024
:1003A000816003C08091C1008E7F8093C100E09185
:1003B0003001F0E0EB5EFE4F848D8093C6008091AB
:1003C00030018F5F8093300180913001883010F0D0
:1003D00010923001FF91EF919F918F910F900FBE7E
:1003E0000F901F9018951F920F920FB60F92112425
:1003F0002F933F938F939F93EF93FF935A9B03C049
:100400008091C60030C0209115018091160130E026
:1004100090E001972817390741F080911501873145
:1004200079F480911601882359F4809116018F5F29
:100430008093160180911601883110F010921601F8
:10044000E0911501F0E08091C600EB5EFE4F8283E3
:10045000809115018F5F809315018091150188317E
:1004600010F010921501FF91EF919F918F913F91A4
:100470002F910F900FBE0F901F901895482FA895A1
:1004800007C08091C10080628093C1007894A895D4
:1004900020912F018091300130E090E001972817E2
:1004A000390779F380912F01873021F48091300151
:1004B000882339F3E0912F01F0E0EB5EFE4F448F8B
:1004C00080912F018F5F80932F0180912F018830C1
:1004D00010F010922F018091C10080628093C100C2
:1004E000842F0895282F5A99FECF80913901806872
:1004F00080933901109216018091160180931501A5
:100500002F77A22FA295AF70B0E0A050BF4FE22F7F
:10051000F0E0EF70F070E050FF4F8C9190818927F0
:10052000822B0E943E0208955A991CC09091150199
:10053000809116019817B1F0E0911601F0E0EB5EA2
:10054000FE4F9281F894809116018F5F809316017F
:1005500080911601883110F010921601292F30E099
:10056000789402C02FEF3FEFC90108958BB190E05E
:10057000969587959695879581700895EF92FF924D
:100580000F931F939C01181619061CF580912603E2
:1005900090912703A0912803B091290379010027A6
:1005A000F7FC0095102FE80EF91E0A1F1B1F809103
:1005B000C100877F8093C1005A9A599A02C00E9455
:1005C0006A00C801B7010E9488118823C1F30E9404
:1005D00076011F910F91FF90EF9008951092C10046
:1005E0001DBA10926800EDE6F0E010828081ECE622
:1005F000F0E08083808180936B0093E09CBB87E078
:100600008BBB1CBC94B915B881E087B98EE388B95F
:100610008EEF8AB99BB90E94FB00A8952EE088E175
:1006200090E00FB6F894A895809360000FBE2093D9
:100630006000089584B1837C84B985B1837C85B9D9
:1006400084EE8CBD01C08EB50DB407FCFCCF0895BF
:100650001F920F920FB60F9211242F933F934F9337
:100660005F936F937F938F939F93AF93BF93EF931A
:10067000FF9380912B0390912C032FEF8F3F9207D4
:1006800079F0249A8EBD0DB406FE03C024980E9412
:10069000C70D8FEF9FEF90932C0380932B0301C026
:1006A00024988EB50E94430E8DB59EB587FDFCCF74
:1006B00086FDFACFFF91EF91BF91AF919F918F91FE
:1006C0007F916F915F914F913F912F910F900FBE4E
:1006D0000F901F9018958091260390912703A09169
:1006E0002803B091290380933A0190933B01A09392
:1006F0003C01B0933D010895809110018F3F09F1B5
:1007000060913A0170913B0180913C0190913D01D3
:100710006115710581059105B1F06C507E4F8F4FC9
:100720009F4F0E948811882371F0409A8FEF809329
:10073000100110923A0110923B0110923C0110926C
:100740003D0180E0089581E0089580E090E060E060
:1007500040E050E00E94C61040988091260390919E
:100760002703A0912803B091290380933A01909325
:100770003B01A0933C01B0933D010895EF92FF929D
:100780000F931F93DF93CF93CDB7DEB760970FB66C
:10079000F894DEBF0FBECDBF7C010E94070DFC01A7
:1007A000D70112962C91129713968C911397082FBC
:1007B00010E01695102F002717950795822F90E0CF
:1007C000082B192B11968C918930D9F08A3030F48E
:1007D000833059F0853009F065C00DC0803209F4CE
:1007E0005FC0833209F05EC016C0822F0E94930062
:1007F00059C00E94B007C8010E940C0D0097C9F7AC
:1008000051C0309709F44EC012830183D70114966A
:100810008C91838347C0F7018581882311F420E000
:1008200001C020E8C80168E070E00E94C911698336
:100830002A83C8018770907083309105F1F084306D
:1008400091054CF481309105A1F0823091059CF422
:10085000892B69F01CC08530910599F08530910590
:1008600074F08630910579F0079789F40EC0216005
:100870000DC022600BC0246009C0286007C0216140
:1008800005C0226103C0246101C028612A8380E27F
:1008900060E042E49E012F5F3F4F0E94890402C046
:1008A0000E94690180912D03882381F0D7012C914A
:1008B00030E02F7730708091100190E028173907D1
:1008C00029F480912D03815080932D0360960FB6FB
:1008D000F894DEBF0FBECDBFCF91DF911F910F9176
:1008E000FF90EF900895FC018181893159F02091AA
:1008F000C2013091C3012115310551F0CF01F90139
:100900000995089584818093C90181E08093C8018D
:100910000895CF93DF93582FE9019091C00182E1B0
:10092000989FF0011124EC5AFE4F652B608342839F
:100930004F70DF01139603C089918D93415044237A
:10094000D9F7503211F481E001C083E081838091B6
:10095000C0018F5F8093C0018091C001863010F08C
:100960001092C0019091C0018091C101981759F473
:100970008091C1018F5F8093C1018091C101863058
:1009800010F01092C101DF91CF910895DF93CF93C2
:10099000CDB7DEB72F970FB6F894DEBF0FBECDBF31
:1009A0000E946700833061F0843061F09E012F5F08
:1009B0003F4F823081F4198280E660E041E80FC049
:1009C00081E001C082E0898380E660E041E69E012B
:1009D0002F5F3F4F04C0198280E660E041E60E942D
:1009E00089042F960FB6F894DEBF0FBECDBFCF910E
:1009F000DF910895DF92EF92FF920F931F93CF93B1
:100A0000DF93EC01062F7A012115310519F42FEF40
:100A10003FEF43C0C9010E94750F9093C3018093BB
:100A2000C201D093C501C093C4011092C8018EEFDA
:100A30009FEF9093C7018093C60110E084E0D82E09
:100A4000002329F080E0602FA7010E945711D09267
:100A50002D0302C00E946A008091C801882321F4FE
:100A600080912D038823B1F70E946D0F811110E052
:100A70008091C801882319F41F5F183008F3809112
:100A8000C2019091C3010E94750F1092C301109290
:100A9000C2012091C6013091C701C901DF91CF91F8
:100AA0001F910F91FF90EF90DF900895EF92FF92CA
:100AB0000F931F93DF93CF9300D000D000D0CDB71A
:100AC000DEB78C017E010894E11CF11C86E0F70181
:100AD00011928A95E9F7F8018385807F8387C701A2
:100AE0000E944B11C8016EE0A70129EF35E00E947A
:100AF000FA0426960FB6F894DEBF0FBECDBFCF9195
:100B0000DF911F910F91FF90EF900895EF92FF9268
:100B10000F931F93DF93CF9300D000D000D0CDB7B9
:100B2000DEB78C01FC01618172817E010894E11CB9
:100B3000F11CC7010E944B11F80164816095607837
:100B400045815681C7010E94341180E063E0A7010E
:100B50000E945711F8016481607845815681C70170
:100B60000E94341180E063E0A7010E94571126968D
:100B70000FB6F894DEBF0FBECDBFCF91DF911F91AE
:100B80000F91FF90EF900895EF92FF920F931F93B4
:100B9000DF93CF9300D000D000D0CDB7DEB78C016B
:100BA000FC01618172817E010894E11CF11CC70186
:100BB0000E944B11F80145815681C70164810E9452
:100BC000341180E063E0A7010E94571188E0F8012A
:100BD000818783858F77838726960FB6F894DEBF4B
:100BE0000FBECDBFCF91DF911F910F91FF90EF907E
:100BF0000895EF92FF920F931F93CF93DF93FC0121
:100C0000C091C401D091C501209721F481E0809367
:100C1000C801BCC08381282F30E03695322F2227AF
:100C200037952795828190E0282B392B8181893057
:100C300081F08A3020F4873008F4A8C011C08D30CC
:100C400009F465C08D3008F4A1C0803108F09EC061
:100C500007C03A83298384818B838B85846094C009
:100C60009581668177818F3011F0883019F48B85FA
:100C700082608AC03A832983392F330F330F20E0F3
:100C8000442737FD4095542F8D819E81AF81B885D3
:100C900080709070282B392B4A2B5B2B862F90E08D
:100CA0008F779070A3E0880F991FAA95E1F7AA2784
:100CB00097FDA095BA2F282B392B4A2B5B2B872F1A
:100CC00090E08077907064E0959587956A95E1F75C
:100CD000AA2797FDA095BA2F282B392B4A2B5B2BDF
:100CE0002D833E834F835887858190E08074907078
:100CF000880F991F2481282B2C832B85822F8160BC
:100D00008B87878180FD51C023602B874EC08481F3
:100D100090E0A0E0B0E08F779070A070B0708C0190
:100D2000FF24EE24268130E040E050E07EE1220FF7
:100D3000331F441F551F7A95D1F78D819E81AF8156
:100D4000B885A070B070282B392B4A2B5B2B2E292D
:100D50003F29402B512B858190E0A0E0B0E08F77B8
:100D60009070A070B07067E1880F991FAA1FBB1F19
:100D70006A95D1F7282B392B4A2B5B2B2D833E8389
:100D80004F8358878B8588608B870FC02091C20165
:100D90003091C3012115310521F0CF01F9010995E9
:100DA0000FC0CF010E94BE030BC08B858F708F30A8
:100DB00039F481E08093C8011092C7011092C601F6
:100DC000DF91CF911F910F91FF90EF900895EF92D7
:100DD000FF920F931F93CF93DF93162FE42E052FCF
:100DE0000E947202812F0E943E02F82E1F702E2D4B
:100DF000302FC901EC0104C089910E943E02F826FF
:100E00009E012E192117C0F38F2D0E943E02DF9103
:100E1000CF911F910F91FF90EF900895DF93CF93A3
:100E2000CDB7DEB72F970FB6F894DEBF0FBECDBF9C
:100E30006D89762F7F70CE014696DC0120E030E090
:100E4000AE014F5F5F4F08C0FA01E20FF31F8C91B4
:100E500080832F5F3F4F12967217B1F78C890E94E3
:100E6000E7062F960FB6F894DEBF0FBECDBFCF9129
:100E7000DF9108951F93CF93DF93182FEB018B81A0
:100E80000E94BF11982F8B3120F08D3120F08E37CA
:100E900021F0A0E003C0A2E001C0A4E08985883071
:100EA00009F0A860EC816E2F6F779B51923078F437
:100EB00061116D5F862F90E08170907074E0880FF3
:100EC000991F7A95E1F766956F70682B02C06111E2
:100ED0006F5F2D813E814F815885C901817090706F
:100EE000892B11F470E001C070E1E0786E2B8DB7B2
:100EF0009EB70A970FB6F8949EBF0FBE8DBFEDB791
:100F0000FEB731961066CDB7DEB7198384EE8183C4
:100F1000A283138264831582DA01C9018E719070F5
:100F2000A070B070B695A79597958795782B768326
:100F3000178215E056954795379527951A95D1F75D
:100F4000208711860E940E078DB79EB70A960FB6AE
:100F5000F8949EBF0FBE8DBFDF91CF911F91089572
:100F60000F931F93DF93CF93CDB7DEB72F970FB6B5
:100F7000F894DEBF0FBECDBF8C010097F1F080E486
:100F80008983F80121813281832F992787FD9A95E2
:100F9000982F8A832436310514F0906C9A83F801D7
:100FA00081818B838081806663EEAE014F5F5F4FEE
:100FB0000E94E70687E0F80182872F960FB6F89423
:100FC000DEBF0FBECDBFCF91DF911F910F9108956E
:100FD000BF92CF92DF92EF92FF920F931F93DF9316
:100FE000CF9300D000D000D0CDB7DEB77C016B012D
:100FF000009709F46BC06115710509F467C0DC0145
:1010000011968D919C91129719962C91861797079E
:1010100019F4283059F458C0283019F487E0F70142
:101020008187D7011296DC92CE921197C6010E9459
:101030000C0DFC01009719F18E159F0501F18181BE
:101040009281D70112969C938E9311978381139668
:101050008C931397848114968C93149725813681F1
:101060004781508515962D933D934D935C9318972A
:10107000CF010E94B00788E0F701828725C0F6E023
:10108000BF2E8E010F5F1F4FD801EB2D1D92EA95E9
:10109000E9F7D7011B968C911B97807F1B968C9349
:1010A000C801B6010E944B11C70161E0A80129EFF8
:1010B00035E00E94FA0497FF03C0F701B28606C02C
:1010C00088E0D7011A968C9381E001C080E02696D3
:1010D0000FB6F894DEBF0FBECDBFCF91DF911F9149
:1010E0000F91FF90EF90DF90CF90BF900895DF9227
:1010F000EF92FF920F931F93DF93CF9300D000D016
:1011000000D0CDB7DEB7AC012FEF8F3F920769F16A
:1011100086E080932A0380913E01882329F410926F
:101120005301109252014EC420915201213168F4B2
:10113000E22FF0E0EF5BFE4F408380915301842764
:10114000809353012F5F209352012091520122304E
:1011500008F438C430E08091410190E08F709070C5
:1011600002962817390709F02DC40E94B602882379
:1011700019F086E080932A0380912A038823E1F006
:1011800011E015C0812F60E00E942C0DFC0100973A
:1011900051F08185883039F4838587FF04C0CF0101
:1011A0000E94C4050FC41F5F1F3109F40BC40E94C5
:1011B000D80D04973CF706C440915201242F30E02B
:1011C0008091410190E08F70907002962817390746
:1011D00009F051C380915301882309F04CC30E9448
:1011E0007F0FD0903E018F3F81F400D000D0EDB74B
:1011F000FEB7319630E6D32AADB7BEB71196DC9272
:1012000081E6818381E890E048C3409A8D2D61E0BA
:101210000E94720D8C01009709F4FCC2FC018185CB
:10122000863081F400D000D0EDB7FEB7319620E6CD
:10123000D22AADB7BEB71196DC9281E6818381E8F0
:1012400090E0F7C2823018F482E0F8018187909133
:101250004101892F82958F70853009F4F2C0863064
:1012600030F4823071F0843009F0D4C275C0893016
:1012700009F449C28E3009F413C1883009F0CAC29A
:1012800009C1903221F4D8011A961C92DAC28091D9
:101290004201843259F1853220F4813209F0B2C220
:1012A00007C0803809F445C0813809F0ABC249C095
:1012B000EDB7FEB738970FB6F894FEBF0FBEEDBF7F
:1012C000319620E6D22AADB7BEB71196DC9283E6FE
:1012D000818381E290E09383828386E390E095832B
:1012E000848381E090E097838683C4C10E94670075
:1012F000823011F421E009C0882311F422E005C0F6
:10130000843011F428E001C020E000D000D000D0EB
:10131000EDB7FEB7319630E6D32AADB7BEB711961A
:10132000DC9282E6818382E290E09383828324834D
:1013300081C00E946700882341F080E060E240E0C5
:10134000ACC00E946700833019F40E94C60479C2C1
:1013500080E060E243E0A1C080914201E82EFF24DA
:10136000EE0CFF1CEE0CFF1C8091430180FF04C0BB
:10137000E2E0F0E0EE0EFF1EE1FC02C010E001C072
:1013800010E181E491E0B7010E944B1180E090E010
:1013900069E141E451E023E734E00E94FA048091DE
:1013A000C901823551F083351CF4873459F408C0E3
:1013B000873639F0823731F401C01068116002C0FD
:1013C00010681260B7016F5F7F4F81E491E00E9467
:1013D0004B1180E090E069E141E451E023E734E023
:1013E0000E94FA048091C901823551F083351CF4C2
:1013F000873459F408C0873639F0823731F401C098
:101400001068146002C01068186000D000D000D0CE
:10141000EDB7FEB7319620E6D22AADB7BEB711962A
:10142000DC9282E48183F694E794F694E794F38265
:10143000E282148315820E940E07EDB7FEB736963E
:101440001EC16091420170E093E0660F771F9A958C
:10145000E1F70091430110E0C80187709070682B9C
:10146000792B81E090E0682779277E010894E11CC0
:10147000F11CC7010E944B111B8283E01695079552
:101480008A95E1F701700C8380E066E0A7010E9475
:101490005711D7C180E060E242E00E946D11D1C1D6
:1014A0009091430180E020914401E22EFF24E82A3C
:1014B000F92A2FEF3FE3E222F322809142018331A8
:1014C000A8F4813108F0E1C0883009F482C0893085
:1014D00030F48823D9F0873009F094C160C0893096
:1014E00009F49DC0803109F08DC1F7C0803209F444
:1014F00015C1813220F4833109F084C1F3C08132F7
:1015000009F43FC1823209F07DC158C1D80111965A
:101510008D919C911297E816F906A1F119968C917C
:101520001997883019F487E019968C93C7010E94A7
:101530000C0DFC010097E9F080179107D1F0818133
:101540009281D80112969C938E9311978381139662
:101550008C931397848114968C9385819681A781AF
:10156000B085F80185839683A783B08787E081875C
:1015700004C0C801B7010E9456058D2DB8010E9414
:101580003A075FC18D2DB8010E943A07D801119624
:101590006D917C911297C8010E94560552C1EDB71A
:1015A000FEB738970FB6F894FEBF0FBEEDBF319669
:1015B00020E6D22AADB7BEB71196DC9283EE8183C6
:1015C00080E590E0938382831582148217821682CD
:1015D00051C02DB73EB72A5030400FB6F8943EBFE9
:1015E0000FBE2DBFEDB7FEB7319630E6D32AADB7AB
:1015F000BEB71196DC9284EE818381E590E09383FF
:10160000828315821482178216828FE090E0918780
:1016100080870E940E07EDB7FEB73A9630C0D8011A
:1016200015964D915D916D917C911897EDB7FEB730
:1016300038970FB6F894FEBF0FBEEDBF319620E687
:10164000D22AADB7BEB71196DC9223EE218322E5F4
:1016500030E033832283BDE07695679557954795B3
:10166000BA95D1F744831582BB27A72F962F852FD4
:10167000868317820E940E07EDB7FEB738960FB625
:10168000F894FEBF0FBEEDBFDCC0C801B7010E94D9
:10169000E807882309F4D5C040914501842F90E0E4
:1016A0009C012071307054E0359527955A95E1F7EB
:1016B0008F709070880F991F282B822F8150823055
:1016C00028F44078D80114964C931DC02111235062
:1016D0004078242BF801248391C0809145018F78B4
:1016E00080934501C801B7010E94E807882309F4E7
:1016F000A8C090914501892F8F77813041F490786F
:10170000D80114969C93C8010E9486059AC0811145
:1017100081509078892BF801848370C0C801B7018B
:101720000E94E807882309F48CC080914501D80104
:1017300015962D913D914D915C91189784FF07C0AE
:101740002160F801258336834783508708C02E7FA8
:10175000D80115962D933D934D935C9318978091E6
:10176000450190E08F709070880F991FAA2797FD10
:10177000A095BA2FF8012581368147815085217EB9
:1017800035C0C801B7010E94E807882309F459C091
:101790008091450190E08F709070B5E0880F991F9F
:1017A000BA95E1F7AA2797FDA095BA2FF8012581F0
:1017B0003681478150852F713E7F18C0C801B7011F
:1017C0000E94E8078823E9F18091450190E08F703D
:1017D0009070982F8827990FAA2797FDA095BA2F68
:1017E000F8012581368147815085317E822B932BEC
:1017F000A42BB52B85839683A783B087C8010E944D
:10180000C4051FC000D000D0EDB7FEB7319620E66A
:10181000D22A07C000D000D0EDB7FEB73196B0E6AF
:10182000DB2AADB7BEB71196DC9281E6818382E8F0
:1018300090E0938382830E940E070F900F900F9089
:101840000F90409880913E0160E00E942C0D8C0129
:10185000009759F1FC018385806883870E94D80D29
:1018600003971CF1D80119968C918830F1F4C801C6
:101870000E94C4051AC04423C1F000D000D0EDB7C7
:10188000FEB7319680913E018066ADB7BEB7119626
:101890008C9381E6818380E890E0938382830E9429
:1018A0000E070F900F900F900F901092530110920F
:1018B000520111E00CE0812F60E00E942C0DFC0130
:1018C000009769F08285882351F0893031F4DF0177
:1018D000202F1D922A95E9F702C0818712861F5F8B
:1018E000103249F70E94B602882309F06BC090912C
:1018F000C0018091C101981729F14091C10182E195
:10190000489F800111240C5A1E4FA8014D5F5F4F64
:10191000D8018C9112966C910E94E706F8018181A2
:1019200081508183882309F04AC08091C1018F5F73
:101930008093C1018091C101863008F440C01092AB
:10194000C1013DC080914001882361F480913F0135
:101950008F5F80933F01803228F010923F0181E039
:101960008093400180913F01882351F060E00E9404
:101970002C0D892B29F480913F0180933E011CC0DE
:1019800080913E010E94800DFC01009751F0808102
:1019900080933E018185863031F4CF010E94B007EB
:1019A00002C010923E01809140018F5F8093400100
:1019B00080913E01882319F080640E94720286E0C3
:1019C00080932A0326960FB6F894DEBF0FBECDBFD4
:1019D000CF91DF911F910F91FF90EF90DF900895CD
:1019E000EAECF1E0482F50E020E030E080818823ED
:1019F00011F421E030E02417350711F480E0089558
:101A00003C9682E0EA38F80779F781E00895809102
:101A10008A0290918B0208959C01EAECF1E00CC0DF
:101A20008285882309F48185883029F48181928117
:101A30008217930739F03C9682E0EA38F80781F77D
:101A4000E0E0F0E0CF01089580ECEAECF1E0DF01A6
:101A50001D928A95E9F70895CF93DF93382F81502F
:101A60008F31D0F5CAECD1E004C088818317B1F181
:101A70002C9682E0CA38D807C1F7662369F120E0C6
:101A8000CAECD1E025C08881882301F5388382E043
:101A9000898700D000D000D0EDB7FEB7319688E638
:101AA00090E0ADB7BEB712969C938E931197328398
:101AB0001382248315820E94F0118DB79EB706967B
:101AC0000FB6F8949EBF0FBE8DBF08C02C962F5F37
:101AD00092E0CA38D907B8F2C0E0D0E0CE01DF9179
:101AE000CF910895882319F420E030E003C00E94CC
:101AF0002C0D9C0130938B0220938A02C90108951A
:101B00000F931F93182F882311F401E005C0803232
:101B100010F00FE101C0082F1F5F103208F011E034
:101B2000812F60E00E942C0D9C01101711F000978E
:101B300099F3C9011F910F91089580E090E00895F5
:101B40008FEF9FEF0895089580E0089580E090E082
:101B500008958FEF9FEF0895DC019091140389E0C1
:101B6000989FF0011124EA56FD4F90E08D918193EA
:101B70009F5F9930D9F7809114038F5F809314038E
:101B800080911403863010F010921403089510927F
:101B900020031092190310921803089590911403D2
:101BA0008091150320E0981709F421E0822F089511
:101BB0008FB7F8949091140320911503492F50E0AA
:101BC000421B51098FBF57FF02C04A5F5F4F25E09C
:101BD00030E0241B350BC90108951F93AC011FB7DA
:101BE000F894209114038091150330E090E0019760
:101BF0002817390741F080911403853039F480911A
:101C00001503882319F41FBF80E005C0CA010E9494
:101C1000AC0D1FBF81E01F910895DC01EDE8F2E0FB
:101C20008D91819382E0E639F807D1F708959C0100
:101C3000009739F14FB7F8949091160380911703EC
:101C4000981721F44FBF20E030E01BC0909117039C
:101C500089E0989FF0011124E453FD4FD90190E0F1
:101C600081918D939F5F9930D9F7809117038F5F92
:101C70008093170380911703883010F01092170398
:101C80004FBFC90108951F93182F87FF86C0809109
:101C9000160390E001969C0143E0220F331F4A9502
:101CA000E1F7280F391F24533D4F80911A0390917B
:101CB0001B0382179307E1F4809116038F5F8093D3
:101CC000160380911603883010F01092160390913D
:101CD000160380911703981759F4809117038F5FAB
:101CE0008093170380911703883010F01092170328
:101CF00010921B0310921A031092190310921803EA
:101D000080911001181721F481E08093200377C09F
:101D100010922003412F50E04F775070682F70E0F1
:101D20004617570729F01F3F19F08F3F09F067C08A
:101D30008091160329E0829FC001112484539D4F96
:101D400090931B0380931A034617570709F057C057
:101D50009091140380911503981721F48DE892E077
:101D60000E94AC0D8091150329E0829FC0011124CF
:101D70008A569D4F90931903809318038091150301
:101D80008F5F8093150380911503863010F01092B9
:101D9000150389E080938C0232C02091200321300A
:101DA00029F0213060F1263050F515C082E0809393
:101DB0002003103419F41092210321C0113419F4B6
:101DC000209321031CC0123419F0133491F483E0E2
:101DD0008093210314C0E22FF0E08091210390E072
:101DE00002968E179F0744F0E65EFC4F808118171D
:101DF00019F01092200303C02F5F209320030E944C
:101E00006700883021F180912003882329F0109306
:101E10002B0310922C0321C0E0911803F0911903B9
:101E20003097A9F0819180932B0310922C03F093AB
:101E30001903E093180380918C02815080938C02E7
:101E4000882359F4109219031092180306C08FEFDB
:101E50009FEF90932C0380932B03E0911A03F09152
:101E60001B03309749F083E0E431F80728F411931D
:101E7000F0931B03E0931A031F9108958FEF9FEFD8
:101E800090932C0380932B030E945A01262F2F77C7
:101E900020931F03F7E09695879577956795FA95B8
:101EA000D1F7262F2F7720931E03E7E0969587958D
:101EB00077956795EA95D1F7262F2F7720931D0305
:101EC00057E096958795779567955A95D1F76F77EF
:101ED00060931C030E941A030895809124038823B1
:101EE00019F01092240381E008952091220330918B
:101EF00023039093230380932203C90108958091C3
:101F000010010895FF920F931F93DF93CF93CDB7E6
:101F1000DEB729970FB6F894DEBF0FBECDBFDA014A
:101F2000A89580911001806889836A83FE013396A9
:101F30009E01275F3F4F109721F08D918F7780830F
:101F400001C010823196E217F307A9F78E010F5FE7
:101F50001F4FC8010E940E118987F02E012F8F2D6F
:101F6000902F0E94ED0D8823D1F381E029960FB6C2
:101F7000F894DEBF0FBECDBFCF91DF911F910F91BF
:101F8000FF9008952F923F924F925F926F927F92AF
:101F90008F929F92AF92BF92CF92DF92EF92FF9279
:101FA0000F931F93DF93CF93CDB7DEB729970FB66B
:101FB000F894DEBF0FBECDBF809110018F3F09F0B6
:101FC0006FC00E945A019B01AC0139014A0177E0C0
:101FD00095948794779467947A95D1F78FE790E0FA
:101FE000A0E0B0E0682279228A229B2259016A018E
:101FF0006EE0D594C794B794A7946A95D1F7A822B8
:10200000B922CA22DB2279018A0195E1159507954B
:10201000F794E7949A95D1F787E090E0A0E0B0E0DC
:10202000E822F9220A231B238FE7282E312C412C8A
:10203000512C222233224422552234C0A8958A8171
:10204000843081F5CE0101960E942511882351F13B
:102050008E8190E0A0E0B0E0281639064A065B06C3
:1020600009F58D8190E0A0E0B0E0681679068A0657
:102070009B06C1F48C8190E0A0E0B0E0A816B90600
:10208000CA06DB0679F48B8190E0A0E0B0E0E816A8
:10209000F9060A071B0731F489818F7780931001B5
:1020A00081E007C0CE0101960E94170E892B31F600
:1020B00080E029960FB6F894DEBF0FBECDBFCF915A
:1020C000DF911F910F91FF90EF90DF90CF90BF9025
:1020D000AF909F908F907F906F905F904F903F90C8
:1020E0002F900895FF920F931F93DF93CF93CDB757
:1020F000DEB729970FB6F894DEBF0FBECDBF809133
:1021000010018F3F69F50E94C20F882399F18091D9
:1021100010010E94A5032EC0C8010E94251188232A
:1021200021F1298130E02F7730708091100190E00B
:102130002817390711F40E946B038A81863019F43D
:10214000F092240312C0E0912203F0912303309710
:1021500019F0C801099509C0C8010E94BE0305C055
:102160008E010F5F1F4FFF24F394C8010E94170ECA
:10217000892B91F629960FB6F894DEBF0FBECDBF1E
:10218000CF91DF911F910F91FF9008950F931F93AF
:10219000DF93CF93CDB7DEB729970FB6F894DEBFA4
:1021A0000FBECDBF209110012068298323E02A8330
:1021B000282F2F772B83880F892F881F990B9195B4
:1021C0008F778C83862F8F778D83852F8695869545
:1021D0008E8367FF02C080648E83CA01E3E0969518
:1021E0008795EA95E1F78F778F83842F82958077A3
:1021F00088878E010F5F1F4FC8010E940E118987CB
:10220000C8010E940D0E29960FB6F894DEBF0FBECE
:10221000CDBFCF91DF911F910F910895FC0120E078
:1022200090E037E08191982780E097FF03C0990FF5
:10223000932701C0990F8F5F8830B9F72F5F28303F
:1022400089F797FD9095892F08950F931F938C011F
:102250000E940E1120E0F8019085891709F421E011
:10226000822F1F910F910895FC01862F8F77828313
:10227000852F8695869566956074862B8383CA0123
:1022800023E0969587952A95E1F78F778483429589
:10229000407745830895FC01862F8F778083660FF2
:1022A000672F661F770B71956F77618308950F9382
:1022B0001F93CF93DF93082F162FEA0102C00E94CD
:1022C0006A00802F612FAE010E94820F8823B9F32C
:1022D000DF91CF911F910F910895DF93CF9300D09D
:1022E00000D000D0CDB7DEB7FE01319696E0DF0119
:1022F0001D929A95E9F74983AF010E9457112696DE
:102300000FB6F894DEBF0FBECDBFCF91DF91089519
:102310009B01AC018091260390912703A091280393
:10232000B091290382179307A407B50798F080910D
:10233000260390912703A0912803B091290360E020
:10234000821B930BA40BB50B80509041A040B04072
:10235000A0F412C08091260390912703A091280336
:10236000B091290360E0281B390B4A0B5B0B20500E
:10237000304F4F4F5F4F08F061E0862F0895E82FF0
:10238000F0E0EF70F070E158FF4FE4918E2F90E095
:10239000089597FB092E07260AD077FD04D00CD0AC
:1023A00006D000201AF4709561957F4F0895F6F7D6
:1023B000909581959F4F0895AA1BBB1B51E107C0C3
:1023C000AA1FBB1FA617B70710F0A61BB70B881FC5
:1023D000991F5A95A9F780959095BC01CD01089554
:1023E000A0E0B0E0E6EFF1E10C94A314FE01359615
:1023F00061917191A0913003B091310313968C914A
:102400001397886013968C938091300390913103D9
:10241000AF010E941612E0913003F0913103238145
:10242000277F23832096E2E00C94BF14ABE0B0E05A
:10243000ECE1F2E10C9493143C012B015A01FC01F4
:1024400017821682838181FD03C06FEF7FEFC6C1C3
:102450009AE0892E1E010894211C311CF30123816E
:10246000F20123FD859123FF81912F01882309F437
:10247000B2C1853239F423FD859123FF81912F016B
:10248000853229F490E0B3010E940914E7CF982F18
:10249000FF24EE249924FFE1FF15D0F09B3269F070
:1024A0009C3228F4903259F0933291F40EC09D3250
:1024B00049F0903369F441E024C052E0F52A84E009
:1024C000F82A28C098E0F92A25C0E0E1FE2A22C0B7
:1024D000F7FC29C0892F80538A3070F4F6FE05C0BE
:1024E000989C902C1124980E15C0E89CE02C112487
:1024F000E80EF0E2FF2A0EC09E3229F4F6FC6BC112
:1025000040E4F42A07C09C3619F450E8F52A02C0CA
:10251000983649F4F20123FD959123FF91912F0103
:10252000992309F0B8CF892F8554833018F0805251
:10253000833038F444E050E0A40EB51E5FE35983C5
:102540000FC0933631F0933779F0933509F056C0C8
:1025500020C0F5018081898342E050E0A40EB51EC1
:10256000610101E010E012C0F501C080D180F6FCED
:1025700003C06FEF7FEF02C0692D70E042E050E0D2
:10258000A40EB51EC6010E94FE138C015FE7F52262
:1025900014C0F501C080D180F6FC03C06FEF7FEF5F
:1025A00002C0692D70E042E050E0A40EB51EC601E5
:1025B0000E94F3138C0150E8F52AF3FE07C01AC0FD
:1025C00080E290E0B3010E940914EA948E2D90E01D
:1025D00008171907A8F30EC0F601F7FC8591F7FE5E
:1025E00081916F0190E0B3010E940914E110EA9417
:1025F000015010400115110579F7EAC0943611F029
:10260000993669F5F7FE08C0F501208131814281D4
:10261000538184E090E00AC0F501808191819C01A2
:10262000442737FD4095542F82E090E0A80EB91E54
:102630009FE6F92257FF09C05095409530952195A6
:102640003F4F4F4F5F4FE0E8FE2ACA01B901A10199
:102650002AE030E00E943514D82ED21840C09537B9
:1026600029F41F2D1F7E2AE030E01DC01F2D197F89
:102670009F3661F0903720F4983509F0ACC00FC058
:10268000903739F0983709F0A6C004C028E030E050
:102690000AC0106114FD146020E130E004C014FD94
:1026A000166020E132E017FF08C0F50160817181FA
:1026B0008281938144E050E008C0F50180819181DE
:1026C000BC0180E090E042E050E0A40EB51EA10104
:1026D0000E943514D82ED2188FE7F82EF122F6FE7C
:1026E0000BC05EEFF522D91438F4F4FE07C0F2FCFB
:1026F00005C08FEEF82202C01D2D01C0192DF4FE79
:102700000DC0FE01ED0DF11D8081803319F499EEAD
:10271000F92208C01F5FF2FE05C003C08F2D867826
:1027200009F01F5F0F2DF3FC14C0F0FE0FC01E1543
:1027300010F09D2C0BC09D2C9E0C911A1E2D06C0D6
:1027400080E290E0B3010E9409141F5F1E15C0F3E0
:1027500004C01E1510F4E11A01C0EE2404FF0FC0DE
:1027600080E390E0B3010E94091402FF1DC001FD47
:1027700003C088E790E00EC088E590E00BC0802F92
:10278000867891F001FF02C08BE201C080E2F7FC85
:102790008DE290E0B3010E94091406C080E390E04E
:1027A000B3010E9409149A94D914C0F3DA94F10188
:1027B000ED0DF11D808190E0B3010E940914DD2030
:1027C000A9F706C080E290E0B3010E940914EA94E0
:1027D000EE20C1F743CEF30166817781CB012B96C2
:1027E000E2E10C94AF14FC010590615070400110BF
:1027F000D8F7809590958E0F9F1F0895FC0161502A
:10280000704001900110D8F7809590958E0F9F1F12
:1028100008950F931F93CF93DF938C01EB018B816E
:1028200081FF1BC082FF0DC02E813F818C819D8165
:102830002817390764F4E881F9810193F983E88363
:1028400006C0E885F985802F0995892B31F48E81A2
:102850009F8101969F838E8302C00FEF1FEFC801F7
:10286000DF91CF911F910F910895FA01AA27283087
:1028700051F1203181F1E8946F936E7F6E5F7F4F4D
:102880008F4F9F4FAF4FB1E03ED0B4E03CD0670FC9
:10289000781F891F9A1FA11D680F791F8A1F911D1C
:1028A000A11D6A0F711D811D911DA11D20D009F46C
:1028B00068943F912AE0269F11243019305D3193AE
:1028C000DEF6CF010895462F4770405D4193B3E097
:1028D0000FD0C9F7F6CF462F4F70405D4A3318F03E
:1028E000495D31FD4052419302D0A9F7EACFB4E0EF
:1028F000A6959795879577956795BA95C9F70097A7
:102900006105710508959B01AC010A2E0694579547
:10291000479537952795BA95C9F7620F731F841F9E
:10292000951FA01D08952F923F924F925F926F9234
:102930007F928F929F92AF92BF92CF92DF92EF924F
:10294000FF920F931F93CF93DF93CDB7DEB7CA1BD0
:10295000DB0B0FB6F894DEBF0FBECDBF09942A88FB
:10296000398848885F846E847D848C849B84AA84A3
:10297000B984C884DF80EE80FD800C811B81AA8130
:10298000B981CE0FD11D0FB6F894DEBF0FBECDBFFB
:08299000ED010895F894FFCF5A
:10299800008080008000008080000080008080002F
:0229A800FF002E
:00000001FF
